:03000000024CCEE1
:0C4CCE0078FFE4F6D8FD758178024D15E2
:101F1F0020000A3C2E2E2E3E004950436F6E6E65F8
:101F2F0063745245510A004950436F6E6E65637476
:101F3F00000A49504E6F41434B210A003E432C5635
:101F4F002C43432CC0E4E0EFF2E5F020D1E8EDEABA
:101F5F00EEEC49500A003E432C4D41432C253032C4
:101F6F0062583A25303262583A25303262583A2553
:101F7F00303262583A25303262583A253032625840
:101F8F002C4D414320E0E4F0E5F10A003E432C568E
:101F9F0045522C20332E3220EEF22025732025734C
:101FAF002CC2E5F0F1E8FF20495020ECEEE4F3EB12
:101FBF00FF0A004D61792032342032303132003146
:101FCF00353A32363A3338003E432C4C442C50527B
:101FDF004F473A2020202020202020202020202082
:101FEF0020202020202020202020202020202020E2
:101FFF0020202020202020202020202020202020D2
:10200F0020202020202020202020202020202020C1
:10201F0020202020202020202CC4E0F2E020EFF010
:10202F00EEF8E8E2EAE828F4E0E9EB290A003E2AB4
:10203F002C312CCEF1EDEEE2EDFBE520EFE0F0E000
:10204F00ECE5F2F0FB20F1E5F2E5E2EEE3EE20E85D
:10205F00EDF2E5F0F4E5E9F1E00A003E412C413004
:10206F00312C2562752E2562752E2562752E2562FF
:10207F00752C495020E0E4F0E5F120E0E4E0EFF2C8
:10208F00E5F0E00A003E412C4130322C2562752EDE
:10209F002562752E2562752E2562752C495020E01C
:1020AF00E4F0E5F120EEF1ED2E20F1E5F0E2E5F0C0
:1020BF00E00A003E412C4130332C2562752E2562FB
:1020CF00752E2562752E2562752C495020E0E4F09F
:1020DF00E5F120F0E5E72E20F1E5F0E2E5F0E00A8A
:1020EF00003E412C4130342C2562752E2562752E11
:1020FF002562752E2562752CCCE0F1EAE020F1E522
:10210F00F2E80A003E412C4130352C2562752E2510
:10211F0062752E2562752E2562752CD8EBFEE70AA7
:10212F00003E2A2C312CC4EEEF2E20EFE0F0E0EC35
:10213F00E5F2F0FB20F1E5F2E5E2EEE3EE20E8ED6B
:10214F00F2E5F0F4E5E9F1E00A003E422C533031BC
:10215F002C2562752CC6E4E0F2FC20E7E0EFF0EEF0
:10216F00F1E020F1EEE5E4E8EDE5EDE8FF20EEF239
:10217F0020F1E5F0E2E5F0E00A003E422C53303268
:10218F002C2562752CCEE1ECE5ED20F120F1E5F088
:10219F00E2E5F0EEEC20E1E5E720EAE2E8F2E0ED3F
:1021AF00F6E8E90A003E422C5330332C2562752C99
:1021BF00CFE5F0E5E7E0EFF3F1EA20EFF0E820EF0D
:1021CF00EEF2E5F0E520F1E2FFE7E820F120F1E59E
:1021DF00F0E2E5F0EEEC0A003E422C5330382C25AD
:1021EF0062752CCCE5E4EBE5EDEDFBE920495020E1
:1021FF00EAE0EDE0EB28E7E0E4E5F0E6EAE020E4F2
:10220F00EE203520F1E5EA290A003E422C53303505
:10221F002C2562752CCAE0EDE0EB20F8E8F0EEEA31
:10222F00EEE2E5F8E0F2E5EBFCEDEEE3EE20EEE1B9
:10223F00ECE5EDE00A003E532C5330362C253032BE
:10224F00625825303262582530326258253032625A
:10225F0058253032625825303262582C4D41432078
:10226F00E0E4F0E5F120F8E8F0EEEAEEE2E5F8E080
:10227F00F2E5EBFCEDEEE3EE20EEE1ECE5EDE00A4E
:10228F00003E454E440A000A44756D7058202020C8
:10229F002020303020303120303220303320303485
:1022AF00203035203036203037203038203039205C
:1022BF003041203042203043203044203045203000
:1022CF0046000A3A003A20000A000A44756D70442D
:1022DF002020202020303020303120303220303369
:1022EF002030342030352030362030372030382021
:1022FF0030392030412030422030432030442030CC
:10230F004520304600457272206B6579005264207B
:10231F00656570726F6D0A005264204D454D0A005D
:10232F00526420436F64650A0057726974652043D5
:10233F006F64650A0044656275674950204F4E0A05
:10234F000044656275674950204F46460A00446550
:10235F0062756755736572204F6E0A00446562752A
:10236F006755736572204F46460A0044656275676C
:10237F004D7367204F6E0A0044656275674D736732
:10238F00204F46460A00436F6E666967206C6F6385
:10239F006B210A00577220656570726F6D0A0020FD
:1023AF005361766520656570726F6D210A00457205
:1023BF0072204D414321004C6F61643E3E002A0064
:1023CF00CEF8E8E1EAE00A00202D202575282575D2
:1023DF00290A003C4130313D003C4130323D003C48
:1023EF004130333D003C4130343D003C4130353DC0
:1023FF00003C21003C5330313D003C5330323D0016
:10240F003C5330333D003C5330353D003C53303866
:08241F003D003C5330363D0046
:0655D100017500017300EA
:10561700C28E438910E4F58B758DB8D2ABD28E223A
:03001B00024C3E56
:104C3E00C0E0C083C082C0D0C28E758B00758DB8A7
:104C4E0020250675A61E75A6E10573D221E57560B1
:104C5E000205750578E578540F7051E574D394010B
:104C6E0040021574D22DE578543F7012D21F906613
:104C7E008EE0600A04F0E0D394B44002D225906630
:104C8E0087E0600204F0906104E0600214F0906628
:104C9E008FE0D394014003E014F03024020576E552
:104CAE0077D394644004D22580020577E572D394BD
:104CBE000140021572D28ED0D0D082D083D0E03295
:1018A600C291C290D2B5C22A7D027C007F07125532
:1018B600B48F28E528646060097D017F6012554F6A
:1018C600D22AE4FDFC7F0B1255B48F28E52830E6BA
:1018D600097D04E4FF125573D22A7D017C007F073F
:1018E6001255B48F28E5287008FD7FFF12554FD298
:1018F6002A302A03126000C288C2A8C2AA758900CB
:10190600124FDC90633FE0B4FA06A3E064CE607B3E
:10191600E4F52874372528F582E43463F583E4F08A
:101926000528E528B443EC90633F74FAF0A374CE1F
:10193600F0A374CCF0906345740AF0E4A3F0A3041A
:10194600F0A3F090633B74FFF0A3F0A3F0E4A3F0E0
:101956009063567403F0E4F528E5282401FFE43388
:10196600FE74372528F582E43463F583E0FD1255CD
:101976002B0528E528C3944340DFE4F5A775A61E8A
:1019860075A6E1907FF0F0A3F080FE90634A7403A1
:10199600F0A374CCF0E4906349F090668CF0A3F069
:1019A600124528C2B5123A34C225125259D22AC259
:1019B6002CC22B9065777408F09062B57424F0E41D
:1019C600A3F090633FE09062B7F0906340E09062CE
:1019D600B8F0906341E09062B9F0906342E09062A3
:1019E600BAF0906343E09062BBF0906344E090628B
:1019F600BCF0757401E4906578F0C226C227C2284F
:101A0600C229202A18AF28FE7D0312460EE4FF12D3
:101A16004AF77E1F7F1FE4FBFDFC12442890668E6A
:101A2600E060037401F0E4906104F0F57690657669
:101A3600F0F57712561775A70775A61E75A6E1D29B
:101A4600AFE4F577906104E070031231C090668FC1
:101A5600E06401701D9080007410F09080A874FFFF
:101A6600F0A3F0A3F0A3F0E490668FF0D22AC22B85
:101A7600C22C908008E0F52830E405D2267410F0D8
:101A8600E52830E508D2289080087420F0E5283053
:101A9600E608D2279080087440F0E576C3940340A8
:101AA60019908002E4F0908001F0908000F0E576D5
:101AB60094064006E4F5761252599080A0E0700331
:101AC6001250D49080B8E0700312505A9080D0E043
:101AD60070031251FD908000E070133026101243FF
:101AE60024906332EFF0D3940040031200369080C6
:101AF60002E07006908000E06005D224021A47C218
:101B060024E4F576906104E06003021A47202A1265
:101B1600906579E0600C7E1F7F21124892E4906503
:101B260079F030281212409F906332EFF0D3940080
:101B36004005E0FF122D58202703021CCB123D9BC7
:101B4600906332EFF07003021A47906376E054BF59
:101B5600247F7003021C26147003021BFE240260FD
:101B660003021C6D202A077E1F7F28124892202E12
:101B760003021CCB90634EE07006906352E06067F0
:101B8600906683E0FF90634EE0B50724906684E09C
:101B9600FE90634FE0B50618906685E0FE906350B0
:101BA600E0B5060C906686E0FE906351E06E603705
:101BB600906352E06F6003021CCB906684E0FF9056
:101BC6006353E06F6003021CCB906685E0FF906371
:101BD60054E06F6003021CCB906686E0FF9063556D
:101BE600E06F6003021CCBC2229065787401F0128C
:101BF600564C757401021CCB90668EE0600374012E
:101C0600F090667BE0FF906378E06F6003021CCB88
:101C160090667BE004F0E4F574906576F0021CCBE8
:101C2600302203021CCB906345E07003021A4790F2
:101C360062B4E06008906356741EF08006906356A6
:101C46007403F0125398D222E4F574906576F090FE
:101C5600668704F0E490667AF0A3F0202A677E1F78
:101C66007F36124892805E90668EE060037401F0C3
:101C7600302252906376E020E74B906378E0FF9045
:101C8600667AE0FE6F600D906682E07007EE146F74
:101C96007033801390667AE004F0906332E0FFD3ED
:101CA600940440031200329060007482F0A3740121
:101CB600F0906378E0906002F07E607F007D031212
:101CC6004EDE021A47202203021DEEE574706E12E4
:101CD6005412EF60237E647F76906477E02404FDDF
:101CE600124EDE906682E07009906356E0F574024B
:101CF6001A47E4F574021A47906687E0D3943C408D
:101D06003C906682E070369062B4E07030906687F0
:101D160004F0124A2EE4906476F0A37412F09066F2
:101D26007BE0906478F0A374FDF090610563A201F6
:101D360090647A63A2017F12123757809812564137
:101D46008F28E528B401159060007483F0E4A3F0B1
:101D56007E607F007D02124EDE021A47E528D3948C
:101D660001401C9060007483F0A37401F0E5282400
:101D7600FEA3F07E607F007D03124EDE021A47E569
:101D86007464016003021A47906576E004F0202A25
:101D9600077E1F7F40124892906576E0FFD394013C
:101DA600400B906356E0941E5003E004F0EFC3949A
:101DB60005400DC222E4906578F012564C021A478F
:101DC6007C667D8390634AE0FAA3E0FB7F02124DB6
:101DD6005A7E647F76906477E02404FD124EDE908E
:101DE6006356E0F574021A47E57464016003021A4B
:101DF60047906578E014604624FE60421470030242
:101E06001EE124046003021A47E4F576202E13909F
:101E160065787404F0906576E05401F075740102FB
:101E26001A479080027410F0E4906578F090657619
:101E360004F075741290668374FFF0021A47906678
:101E460083E07003021ECB9064767480F090647811
:101E56007401F0E4A3F0A304F0A37430F0A3747B40
:101E6600F0E4F528747D2528F582E43464F583745E
:101E76007DF0747E2528F582E43464F583E4F0E58C
:101E8600282407906477F07C667D8390634AE0FAA5
:101E9600A3E0FB7F02124D5A7E647F76E528240973
:101EA600FD124EDE906682E0601B125398D222E449
:101EB600F574906576F090668704F0E490667AF0A3
:101EC600A3F0021A47302E07E4906578F08006905A
:101ED60065787404F0757412021A479080027410C3
:101EE600F0757403906576E06401FFF09065787490
:101EF60001F0EF7012906352E0600C12103F906692
:101F060083121057021A4790634E12103F90668351
:081F1600121057021A4780FE69
:011F1E0022A0
:10003600906377E0B444047F0180027F009063768A
:10004600E0B447047E0180027E00EE5F604A906362
:100056003FE0906378F0906340E0906379F09063BE
:1000660041E090637AF0906342E090637BF09063A6
:1000760043E090637CF0906344E090637DF090638E
:10008600777452F09062AE63A2019080A863A201D9
:100096007F06123757020913906332E0C394085063
:1000A6000302091C90633FE0FF906378E06F6003F2
:1000B60002091C906340E0FF906379E06F600302E1
:1000C600091C906341E0FF90637AE06F60030209C8
:1000D6001C906342E0FF90637BE06F600302091CA3
:1000E600906343E0FF90637CE06F600302091C901D
:1000F6006344E0FF90637DE06F600302091C906338
:1001060077E06444701A9080A8E0B4FF139062AE62
:1001160063A2019080A863A2017F06123757801060
:100126009062B2E09080ACF09062B3E09080ADF067
:1001360090668EE060037401F090668F7464F090B0
:1001460063777452F0906376E0646D60030202BADE
:100156007BFF7A1F794B12294B7BFF7A1F796590BB
:10016600633FE0F535A3E0F536A3E0F537A3E0F508
:1001760038A3E0F539A3E0F53A12294B7535FF753A
:10018600361F7537C27538FF75391F753ACE7BFF36
:100196007A1F799B12294B7BFF7A1F79D712294B3D
:1001A6007BFF7A20793D12294B7BFF7A20796A9072
:1001B6006345E0F535A3E0F536A3E0F537A3E0F5B2
:1001C6003812294B7BFF7A20799490634EE0F535FF
:1001D600A3E0F536A3E0F537A3E0F53812294B7B0B
:1001E600FF7A2079C2906352E0F535A3E0F536A395
:1001F600E0F537A3E0F53812294B7BFF7A2079F03A
:1002060090633BE0F535A3E0F536A3E0F537A3E0D0
:10021600F53812294B7BFF7A217913906337E0F585
:1002260035A3E0F536A3E0F537A3E0F53812294B00
:100236007BFF7A21793012294B7BFF7A217959A2EB
:100246002EE433F53512294B7BFF7A2179899066A6
:1002560082E0F53512294B7BFF7A2179B490668EC0
:10026600E0F53512294B7BFF7A2179E79062B4E0FD
:10027600F53512294B7BFF7A227919A220E433F552
:100286003512294B7BFF7A22794590667CE0F5355D
:10029600A3E0F536A3E0F537A3E0F538A3E0F5399A
:1002A600A3E0F53A12294B1238657BFF7A22799042
:1002B60012294B22906376E0644C70737E227F96FF
:1002C600FBFDFC12442890637EE0F529A3E0F52AA5
:1002D600E4F52CE529906380F0A3E52AF07E227FE1
:1002E600D17C637D807B02124428E4F52B852A822B
:1002F600852983E0FF7480252BF582E43463F5833A
:10030600EFF0052AE52A70020529052BE52BB41026
:10031600DC7E227FD47C637D807B10124428052CF2
:10032600E52CC3941040AC7E227FD71248922290CF
:100336006376E0646C7060F52D7E227FD9FBFDFC50
:10034600124428E4F52CE4906380F0A3E52DF07EBA
:10035600227FD17C637D807B02124428E4F52BA8A2
:100366002DE6FF7480252BF582E43463F583EFF0E8
:10037600052D052BE52BB410E67E227FD47C637D0C
:10038600807B10124428052CE52CC3940840B77EC8
:10039600227FD712489222906376E0644B7061F513
:1003A6002B7468252BF582E43463F583E0603274A0
:1003B60068252BF582E43463F583E0F460237468E2
:1003C600252BF582E43463F583E0FF747E252BF557
:1003D60082E43463F583E0B50710052BE52BB408FA
:1003E600C09061047432F00209139063767421F0B0
:1003F600302A030209137E237F141248920209133E
:10040600906376E0B4521A202A077E237F1C124896
:10041600929063767472F07E637F767D08124E5EEC
:1004260022906376E064497045202A077E237F2761
:1004360012489290637EE0F529A3E0F52AE4F52BB5
:10044600852A82852983E0FF7480252BF582E43492
:1004560063F583EFF0052AE52A70020529052BE5E9
:100466002BB480DC7E637F767D8A124E5E2290639B
:1004760076E064437046202A077E237F2F12489237
:1004860090637EE0F529A3E0F52AE4F52B852A8220
:10049600852983E493FF7480252BF582E43463F584
:1004A60083EFF0052AE52A70020529052BE52BB412
:1004B60080DB7E637F767D8A124E5E22906376E0D5
:1004C600645A7053202A077E237F3812489290631D
:1004D6007EE0F529A3E0F52A7C637D807B80AF2A48
:1004E600AE291254F7E4F52B852A82852983E493F5
:1004F600FF7480252BF582E43463F583EFF0052A3B
:10050600E52A70020529052BE52BB480DB7E637F87
:10051600767D8A124E5E22906376E0644460030222
:1005260005AE90637EE0FF64447003020913EFB4E6
:10053600310CC22A7E237F4412489202091390632B
:100546007EE0B4300CD22A7E237F501248920209F4
:100556001390637EE0B4320CD22B7E237F5D12486B
:100566009202091390637EE0B4330CC22B7E237F84
:100576006B12489202091390637EE0B4340CD22CBD
:100586007E237F7A12489202091390637EE0B43587
:100596000CC22C7E237F8712489202091390637E39
:1005A600E0FF12001E020913906104E07013202A76
:1005B600077E237F951248929063767421F0020994
:1005C600139061047432F0906376E0FFB45104C274
:1005D600AF80FEEF64577045202A077E237FA31263
:1005E600489290637FE0906332F0E4F52B9063329B
:1005F600E0FFE52BC39F40030209137480252BF50A
:1006060082E43463F583E0FF90637EE0252B24AD1E
:10061600F582E43461F583EFF0052B80D0906376A4
:10062600E0645360030206D1202A077E237FAE12C0
:10063600489290633FE0FF9061B6E06F703C906334
:1006460040E0FF9061B7E06F7030906341E0FF904B
:1006560061B8E0B50724906342E0FF9061B9E0B568
:100666000718906343E0FF9061BAE0B5070C90630A
:1006760044E0FF9061BBE06F60169063767421F0F2
:10068600302A030209137E237FBD12489202091302
:10069600E4F52BE4F577AF2BFE74AD252BF582E45C
:1006A6003461F583E0FD12552B052BE52BC394FE33
:1006B60040E1C2AFE4907FF0F0A3F0907FFD74AA12
:1006C600F0A374FFF0A37455F080FE906376E064A7
:1006D6004F705690637EE0F529A3E0F52AE52A459A
:1006E60029700A202A077E237FC6124892202A07ED
:1006F6007E237FCD124892E4F52B7480252BF5825C
:10070600E43463F583E0852A82852983F0052AE5AA
:100716002A70020529052BE52BB480DE90668CE451
:1007260075F080120ECA020913906376E064457074
:100736007490637EE0FEA3E0FF907FF0EEF0A3EFFF
:10074600F0D39400EE94044038907FF0E0FEA3E0EE
:10075600FF90668CE0FCA3E0FD9FEC9E4023E42F17
:10076600FFEE3401FED3ED9FEC9E5015C2AF907F95
:10077600FD74AAF0A374FFF0A37455F0E4F5A78006
:10078600FE7E237FCF1248927BFF7A2379D7907F14
:10079600F0E0F535A3E0F53690668CE0F537A3E09A
:1007A600F53812294B906376E06465600302091CF4
:1007B60090637EE0FFA3E0907FF0CFF0A3EFF0E43C
:1007C600F529F52AD3907FF1E0952A907FF0E09500
:1007D600294020E4F577252AFFE5293401FE852AFC
:1007E60082852983E0FD12552B052AE52A7002052C
:1007F6002980D17E237FE2124DDEEF4E602012006B
:1008060003906345EFF0120003906346EFF0120089
:1008160003906347EFF0120003906348EFF07E23E6
:100826007FE8124DDEEF4E602012000390634EEF1C
:10083600F012000390634FEFF0120003906350EF45
:10084600F0120003906351EFF07E237FEE124DDE2F
:10085600EF4E6020120003906352EFF012000390F7
:100866006353EFF0120003906354EFF0120003900D
:100876006355EFF07E237FF4124DDEEF4E602012BB
:10088600000390633BEFF012000390633CEFF0121D
:10089600000390633DEFF012000390633EEFF07E9D
:1008A600237FFA124DDEEF4E60201200039063376D
:1008B600EFF0120003906338EFF0120003906339F3
:1008C600EFF012000390633AEFF0E4F52BE4F577CE
:1008D600E52B2401FFE433FE7437252BF582E4343F
:1008E60063F583E0FD12552B052BE52BC39443409E
:1008F600DCC2AFE4907FF0F0A3F0907FFD74AAF025
:10090600A374FFF0A37455F0E4F5A780FE7E637F21
:06091600767D08124E5E22
:01091C0022B8
:1054BF00AE07EEC39430400BEED394395005EE2473
:1054CF00D0FF22EEC39461400BEED394665005EEED
:1054DF0024A9FF22EEC39441400BEED3944650050E
:0854EF00EE24C9FF22AF0622E2
:1055ED009062ACE475F001120ECA9062ACE0FEA3BD
:0655FD00E0FF12559722A9
:100003001255ED1254BFEFC454F0FEC0061255ED65
:080013001254BFD0E02FFF22C0
:1051A000E4906CD4F01255ED906CD5EFF0C39430D0
:1051B0004018E0FFD394395011906CD4E02405F5E9
:1051C00082E43461F583EFF08011906CD4E0240523
:1051D000F582E43461F583E4F0800C906CD4E00453
:1051E000F0E0D3940840BE7532007533007534008A
:0C51F000E4F5357B017A617905123BF78C
:0151FC002290
:044DDE008E2F8F3055
:104DE2009062ACE4F0A374FFF01255EDEF6069F449
:104DF2006066853082852F83E493B507EC753101B7
:104E0200E5302531F582E4352FF583E49360259072
:104E120062ADE02531FF9062ACE03400FE1255979E
:104E2200E5302531F582E4352FF583E493B50704A7
:104E3200053180CCE5302531F582E4352FF583E468
:104E42009370A6E53124FFFFE434FF9062AC8FF04B
:0B4E5200120ECA7E007F0122E4FEFF6A
:014E5D002232
:104528007E247F00124DDEEF4E70037F01227E2431
:104538007F03124DDEEF4E600C1255EDEF24D024B0
:10454800FF922E8002D22E7E247F09124DDEEF4E7E
:10455800600C1255EDEF24D0906682F08005E4904F
:104568006682F07E247F0F124DDEEF4E600C1255EE
:10457800EDEF24D090668EF08005E490668EF07E94
:10458800247F15124DDEEF4E600C1255EDEF24D04E
:1045980024FF92208002C2207E247F1B124DDEEF72
:1045A8004E600C1255EDEF24D09062B4F08005E413
:1045B8009062B4F090633F63A20190667C63A201AD
:1045C8007F0612375730203B7E247F21124DDEEFC5
:1045D8004E603012000390667CEFF0120003906684
:1045E8007DEFF012000390667EEFF01200039066F4
:1045F8007FEFF0120003906680EFF01200039066E0
:0646080081EFF07F0022AB
:10530B00906577E0C3947C40027F0A906577E0FE5E
:10531B0004F074B52EF582E43462F583EFF0BF0A26
:10532B0027906577E0FF04F074B52FF582E43462C3
:10533B00F583E4F0906577E0FF124F5E906577742C
:09534B0008F09062B6E004F022C3
:105259009080007480F090633763A201F583F58232
:1052690063A2017F0812375790633F63A2019080C0
:105279008863A2017F0A1237579080927407F0A3BE
:1052890074D0F0A37406F0906349E0FF9080B1F008
:105299009080E1EFF09080957455F0A3F090800034
:0A52A9007401F090800974F0F02207
:1050D400908009E04410F09080A0E070609080A17E
:1050E4007482F09080A874FFF0A3F0A3F0A3F07F83
:1050F400039080AEEFF0A374CBF09080007402F0C4
:10510400906CDA12106300000000906CDAE090807A
:1051140040F0906CDBE0908041F0906CDCE090809B
:1051240042F0906CDDE0908043F0A3E4F0A3F0A3A0
:0D513400F0A3F0908018F0A3F0A3F0A3F01A
:01514100224B
:1051FD00908009E04440F09080D17482F07F03905C
:10520D0080DEEFF0A374CCF09080027402F0906C0D
:10521D00DE12106300000000906CDEE0908058F00C
:10522D00906CDFE0908059F0906CE0E090805AF047
:10523D00906CE1E090805BF0A3E4F0A3F0A3F0A309
:0B524D00F0908030F0A3F0A3F0A3F07D
:015258002233
:10505A00908009E04420F09080B8E0706C9080B9AC
:10506A007482F07F039080C6EFF07FCDA3EFF07FCC
:10507A00039080C4EFF0A374CDF09080C074FFF069
:10508A00A3F0A3F0A3F09080017402F0906CE212F6
:10509A00106300000000906CE2E090804CF0906C8D
:1050AA00E3E090804DF0906CE4E090804EF0906CDC
:1050BA00E5E090804FF0A3E4F0A3F0A3F0A3F09012
:0950CA008024F0A3F0A3F0A3F090
:0150D30022BA
:104D5A008C298D2AA907EAFDE975F018A424ACFF6D
:104D6A00E5F034808F82F583EDF0EBFDE975F018FC
:104D7A00A4FFAEF024ACFBEE34808B82F583A3ED66
:104D8A00F0852A828C83E0FDEF24A8FFEE3480FEB2
:104D9A008F82F583EDF0852A828C83A3E08F828E41
:104DAA0083A3F0852A82852983A3A3E0FDE975F010
:104DBA0018A424A8FFE5F03480FE8F82F583A3A30C
:104DCA00EDF0852A828C83A3A3A3E08F828E83A32E
:044DDA00A3A3F0227D
:064E5E008D2EAB07AA0631
:104E6400908000E030E5079065797401F022906C41
:104E7400DA12103F8F328E318D308C2FAE02AF0399
:104E84008E838F8263A201E531540744C0F5838584
:104E9400328263A201AF2E1237C9E4FCFDFEE53273
:104EA400252EF532EE3531F531ED3530F530EC3572
:104EB4002FF52F908040E52FF0A3E530F0A3E531E6
:104EC400F0A3E532F09080007420F0AF32AE31AD43
:094ED40030AC2F906CDA1210577B
:014EDD0022B2
:064EDE008D29AB07AA06B6
:104EE400908002E030E5079065797403F022906CBD
:104EF400DE12103F8F2D8E2C8D2B8C2AAE02AF0329
:104F04008E838F8263A201E52C540744D0F58385F8
:104F14002D8263A201AF291237C9E4FCFDFEE52D01
:104F24002529F52DEE352CF52CED352BF52BEC350F
:104F34002AF52A908058E52AF0A3E52BF0A3E52C66
:104F4400F0A3E52DF09080027420F0AF2DAE2CADCF
:094F54002BAC2A906CDE12105700
:014F5D002231
:024AF7008F31FD
:104AF900908001E030E5099065797402F07F002229
:104B0900906CE212103F8F358E348D338C32906663
:104B19007C63A201E534540744C8F5838535826373
:104B2900A2017F061237DFE5352406F535E4353471
:104B3900F534E43533F533E43532F53290657A638B
:104B4900A201E534540744C8F58385358263A2017F
:104B5900AF311237DFE4FCFDFEE5352531F535EEE1
:104B69003534F534ED3533F533EC3532F5329080A3
:104B79004CE532F0A3E533F0A3E534F0A3E535F0D5
:104B89009080017420F0AF35AE34AD33AC32906C07
:064B9900E2121057AF31DB
:014B9F0022F3
:104324009081E0E0F52905290529052905290529B4
:1043340005290529052905290529908010E0F52C72
:10434400A3E0F52DA3E0F52EA3E0F52F9081E1E0A5
:10435400F5290529052905290529052905290529F9
:10436400052905290529908014E0F530A3E0F531ED
:10437400A3E0F532A3E0F533E532B52E08E533B515
:104384002F037F0022E4F529E532540744E0F58346
:1043940085338263A20190637663A2017F08123899
:1043A4000F90637863A2019062AE63A2017F06124C
:1043B4003757906376E0F52AA3E0F52BE4F52990CE
:1043C4006376E0702AA3E024F8F529E53254074423
:1043D400E0F58385338274082582F582E43583F51C
:1043E4008363A20190637663A201AF2912380FAEF2
:1043F4002AE4FCFDE533252BF533E5323EF532EDB9
:104404003531F531EC3530F530908014E530F0A3DA
:10441400E531F0A3E532F0A3E533F0908000744079
:03442400F0AF29CD
:014427002272
:103D9B009081E6E0F529052905290529052905293D
:103DAB0005290529052905290529908028E0F52CE9
:103DBB00A3E0F52DA3E0F52EA3E0F52F9081E7E02E
:103DCB00F529052905290529052905290529052988
:103DDB0005290529052990802CE0F530A3E0F53164
:103DEB00A3E0F532A3E0F533E4F529E532B52E0A6D
:103DFB00E533B52F05C227023F07E532540744F0E0
:103E0B00F58385338263A20190637663A2017F08F9
:103E1B0012380F906376E0F52AA3E0F52BE52B45DE
:103E2B002A70099080027410F07F0022906683E064
:103E3B00FFF46030906378E06F6003023ECE9066D3
:103E4B0084E0FF906379E06F7079906685E0FF9076
:103E5B00637AE06F706D906686E0FF90637BE06F36
:103E6B006031805F906378E0906683F0906379E0D7
:103E7B00906684F090637AE0906685F090637BE0C7
:103E8B00906686F090637CE0FFA3E090634ACFF0EE
:103E9B00A3EFF0906376E0702AA3E024F8F529E510
:103EAB0032540744F0F58385338274082582F582FA
:103EBB00E43583F58363A20190637663A201AF2996
:103ECB0012380FAE2AE4FCFDE533252BF533E53232
:103EDB003EF532ED3531F531EC3530F530AF2FAEF7
:103EEB002EAD2DAC2CAB33AA32A931A830D3121086
:103EFB002E40099080027410F07F002290802CE5F8
:103F0B0030F0A3E531F0A3E532F0A3E533F0908078
:063F1B00027440F0AF2922
:013F2100227D
:10409F009081E3E0F5290529052905290529052939
:1040AF000529052905290529052990801CE0F52CEE
:1040BF00A3E0F52DA3E0F52EA3E0F52F9081E4E02A
:1040CF00F529052905290529052905290529052981
:1040DF00052905290529908020E0F530A3E0F53169
:1040EF00A3E0F532A3E0F533E4F529E532B52E0A66
:1040FF00E533B52F05C2280241F5E532540744E8F0
:10410F00F58385338263A20190600463A2017F0E61
:10411F00123825906004E0F52AA3E0F52B90600C8F
:10412F00E0FFF4604A90667CE0FEEF6E7079A3E0EA
:10413F00FF90600DE06F706F90667EE0FF90600EF5
:10414F00E06F706390667FE0FF90600FE06F7057D5
:10415F00906680E0FF906010E06F704B906681E09A
:10416F00FF906011E06F703FE4906013F080089053
:10417F00601374FFF0D2D9906004E0702AA3E0249A
:10418F00F2F529E532540744E8F583853382740E3E
:10419F002582F582E43583F58363A2019060046381
:1041AF00A201AF29123825AE2AE4FCFDE533252BF9
:1041BF00F533E5323EF532ED3531F531EC3530F58D
:1041CF0030AF2FAE2EAD2DAC2CAB33AA32A931A808
:1041DF0030D312102E5006E52B452A70099080011E
:1041EF007410F07F0022908020E530F0A3E531F0CD
:1041FF00A3E532F0A3E533F09080017440F0AF29CE
:01420F00228C
:044892008E2E8F2FA8
:10489600908000E030E5079065797401F022906C15
:1048A600DA12103F8F358E348D338C32E535FFE5C5
:1048B600345407FEE42FF531EE34C0F530853182ED
:1048C600F5837423F00531E531700205305330C7A6
:1048D600F582853083740AF00531E53170020530C2
:1048E6005330C790633F63A201853083853182636D
:1048F600A2017F061237C974062531F531E4353039
:10490600F530852E83852F8263A20185308385311C
:104916008263A2011237ADE4FCFDFE906CDA121040
:104926004B120F45EF2408FFE43EFEE43DFDE43C58
:10493600FC906CDA121057906CDAE0908040F090A0
:104946006CDBE0908041F0906CDCE0908042F0906F
:0D4956006CDDE0908043F09080007420F054
:014963002231
:0A4428008E318F328C338D348B35CA
:10443200908000E030E5079065797401F022906C7D
:10444200DA12103F8F3B8E3A8D398C38E53BFFE50F
:104452003A5407FEE42FF537EE34C0F5368537823D
:10446200F5837423F00537E537700205365336C7F6
:10447200F582853683740AF00537E5377002053612
:104482005336C790633F63A20185368385378263C3
:10449200A2017F061237C974062537F537E435368F
:1044A200F53685318385328263A20185368385376D
:1044B2008263A2011237AD8F3CEF2537F537E43521
:1044C20036F536E535601785338385348263A2017C
:1044D20085368385378263A201AF351237C9E53C41
:1044E20024082535F535FFE4FCFDFEE53B2FF53BC1
:1044F200EE353AF53AED3539F539EC3538F538908F
:104502008040E538F0A3E539F0A3E53AF0A3E53BB6
:10451200F09080007420F0AF3BAE3AAD39AC3890E9
:054522006CDA121057D5
:014527002271
:0647BE008E2B8F2C8D2DC7
:1047C400908000E030E5079065797401F022906CE8
:1047D400DA12103F8F338E328D318C30E533FFE5A2
:1047E400325407FEE42FF52FEE34C0F52E852F82C8
:1047F400F5837423F0052FE52F7002052E532EC781
:10480400F582852E83EBF0052FE52F7002052E53DC
:104814002EC790633F63A201852E83852F8263A2F6
:10482400017F061237C97406252FF52FE4352EF5BE
:104834002E852B83852C8263A201852E83852F826E
:1048440063A201AF2D1237C97408252DF52DFFE49D
:10485400FCFDFEE5332FF533EE3532F532ED35311F
:10486400F531EC3530F530908040E530F0A3E5319A
:10487400F0A3E532F0A3E533F09080007420F0AFAC
:0D48840033AE32AD31AC30906CDA1210570B
:014891002204
:024F5E008F4E74
:104F6000908000E030E5079065797401F022906C44
:104F7000DA12103F8F528E518D508C4FE552FFE563
:104F8000515407FEE42FFFEE34C09062B563A201D6
:104F9000F5838F8263A201AF4E1237C9E4FCFDFE98
:104FA000E552254EF552EE3551F551ED3550F5509F
:104FB000EC354FF54F908040E54FF0A3E550F0A35E
:104FC000E551F0A3E552F09080007420F0AF52AEAE
:0B4FD00051AD50AC4F906CDA1210573E
:014FDB0022B3
:06460E008E298F2AAB0586
:10461400908000E030E5079065797401F022906C99
:10462400DA12103F8F308E2F8D2E8C2DE530FFE562
:104634002F5407FEE42FF52CEE34C0F52B852C8285
:10464400F5837423F0052CE52C7002052B532BC73E
:10465400F582852B83EBF0052CE52C7002052B905D
:10466400633F63A201852B83852C8263A2017F06AD
:104674001237C97406252CF52CE4352BF52B532B56
:10468400C7E529852C82852B83F0052CE52C700247
:10469400052B532BC7F582852B83E52AF0052CE5E2
:1046A4002C7002052B532BC7E530240AF530E43572
:1046B4002FF52FE4352EF52EE4352DF52D90804081
:1046C400E52DF0A3E52EF0A3E52FF0A3E530F0905F
:1046D40080007420F0AF30AE2FAD2EAC2D906CDA8C
:0346E4001210575A
:0146E70022B0
:0A563600E4FEEEC39F50030E80F85F
:015640002247
:10559700A2AF922FC2AF438E2075D2028F828E8325
:0C55A700E0FFE4F5D2538EDFA22F92AF9C
:0155B30022D5
:10552B00E5D220E0FBA2AF922FC2AF43D2028F8213
:10553B008E83EDF075D25063D250A22F92AFE5D28D
:03554B0020E0FB62
:01554E00223A
:104FDC00E4FDED2401FFE433FE12559774372DF5F3
:104FEC0082E43463F583EFF00DBD3FE6E4FDED2480
:104FFC007FFFE433FE125597742D2DF582E4346156
:10500C00F583EFF0742D2DF582E43461F583E070B7
:10501C001B742D2DF582E43461F5837420F0742E0D
:10502C002DF582E43461F583E4F080040DBD80BE7F
:10503C00E49061ACF0FDEDFF7E0012559774AD2D40
:0D504C00F582E43461F583EFF00DBDFEE95F
:015059002234
:0254F7008B2EFA
:1054F900A2AF922FC2AF85A22F53A2FE8E838F82B5
:1055090005A28C838D827409123853E52E53A2FEAD
:1055190043A22012385553A2DF852FA2A22F92AFA2
:01552900FF82
:01552A00225E
:1055B400A2AF922FC2AF8C838D82EF12385343A2D5
:0C55C4002012385553A2DFA22F92AFFF37
:0155D00022B8
:02554F008F29A2
:10555100A2AF922FC2AFE4F5838D82740612385345
:10556100E52943A22012385553A2DFA22F92AF7F23
:015571000138
:015572002216
:025573008F297E
:10557500A2AF922FC2AFE4F5838D82740A1238531D
:10558500E52943A22012385553A2DFA22F92AF7FFF
:015595000114
:0155960022F2
:10367C00A907E7FFA805EF93C3966008403B74FCCD
:10368C002FFF80F00F08EF93C3966008402B74FB5C
:10369C002FFF80E00F08EF93C3966008401B74FA6D
:1036AC002FFF80D00F08EF93D3966008400B74F96E
:1036BC002FFF80C01F1F1F1F1FEF54FEF80303F7BF
:1036CC00E893FC08E893FD08E893FE08E893FF22D2
:1036DC0009E993C39D6008402974FB29F980F1091D
:1036EC00E993C39E6008401A74FA29F980E209E94B
:1036FC0093D39F6008400B74F929F980D3191919D9
:10370C001919E9C313C313FF22740093F8ECC3987F
:10371C004024701F740193F8EDC398401970147411
:0E372C000293F8EEC398400E7009740393F8F0
:10373A00EFC39840037F00227F0122EDF8E6F008EC
:10374A00A3DFFA22EDF8E0F608A3DFFA22E0A3638A
:10375A00A201F0A363A201DFF475A2002263A20111
:10376A00F0A363A20122E0A363A201F0A363A20172
:10377A00E0A363A201F0A363A201E463A201F0A3A0
:10378A0063A201DFE175A20022E0A363A2016DFE3C
:10379A00936CFDEE058393FC158363A201DFEA7542
:1037AA00A200227F00E493A363A201F00F600CA39E
:1037BA00E583C2E3F58363A20180EA75A20022E0F1
:1037CA00A363A201F0A3E583C2E3F58363A201DF49
:1037DA00EE75A20022E0A363A201F0A3E583C2E48E
:1037EA00D2E3F58363A201DFEC75A20022E0A363B2
:1037FA00A201F0A3E58344F8C2E5F58363A201DFE1
:10380A00EC75A20022E583C2E3F583E0A363A2017B
:10381A00F0A363A201DFEE75A20022E583C2E4D21F
:0A382A00E3F583E0A363A201F0A31D
:1038340063A201DFEC75A20022E58344F8F583E07E
:10384400A363A201F0A363A201DFEE75A20022F933
:1038540022C002C004C00612FFF0D006D004D00279
:013864002241
:10001E00BF360BD20EE4F553F554F56FF570BF37BE
:04002E0002C20E22DA
:10514200C2A9438902906BCFE0FFF58C8F8A75D993
:105152000475DA4875DB3175DC4975DD4975DE3178
:10516200E4F5E9F5F9F5EBF5FB906BCDE06016752A
:10517200EC1075ED10E4F5FCF5FD756B0875691022
:10518200756A01801375EC8075ED80E4F5FCF5FD20
:0E519200756B80F569756A10E4F5EEF5FE2286
:10548600E4FEAF8CEFFD906BCEE07003A3E06D60A1
:10549600051251427E01E5D920E2057E02125142F3
:1054A600E58920E1051251427E03D28C75D84075FC
:0854B600B740D2AED2AFAF0641
:0154BE0022CB
:03003300023F2267
:0B3F2200C0E0C083C082C0D075D00892
:103F2D00C2AF30DC56C3E5EC95EEC3956B5012E590
:103F3D006A25ECF5EC30D70405FC801685FCFC8079
:103F4D0011C3E5EC956AF5EC30D70415FC800385BB
:103F5D00FCFC300E24855482855383E590F0055486
:103F6D00E55470020553F582855383E5EEF0055453
:103F7D00E5547002055353530FC2DC30D929300E6E
:103F8D0024855482855383E590F00554E5547002E1
:103F9D000553F582855383E5EBF00554E554700226
:103FAD00055353530FC2D930DA69E569700405FC26
:103FBD008010E56925ECF5EC30D70405FC80038510
:103FCD00FCFC300F4CE5555480FFE55525E0F555CB
:103FDD003097020555200D03635501303819E5550D
:103FED0054C06571702BEF7028756C08F567855599
:103FFD0058F555C238801A056CE56C54077012538C
:10400D006C3FE56C131313541F2457F8A6557555C3
:10401D0000C2DA30DB71E569700405FD8010E569D9
:10402D0025EDF5ED30D70405FD800385FDFDE56D2E
:10403D0065686029E56854077013E5681313135418
:10404D001F245FF8E6F556200B036356FFE5563344
:10405D009296E55625E0F556056853683FB29230C5
:10406D000E23855482855383E590F00554E55470F5
:10407D00020553F582855383E4F00554E55470022F
:09408D00055353530FC2DBD2AFFF
:09409600D0D0D082D083D0E032FA
:102427000ACFF0E8EDFFF220F6E8EAEBE8F7E5F18E
:10243700EAE8E920EFE0EAE5F220D2D120000ACF6E
:10244700F0E8EDFFF220D2D120F1EE20E2F0E5EC4A
:10245700E5EDE5EC20000ACFF0E8EDFFF220F6E825
:10246700EAEBE8F7E5F1EAE8E920EFE0EAE5F22050
:10247700D2C8D220EEF220E1EBEEEAE02020000AFB
:10248700CEF2E2E5F220EDE020E7E0EFF0EEF1201A
:10249700D2D30A000AC4E0FE20EAEEECE0EDE4F352
:1024A70020E8F1EFEEEBEDE8F2FC20D2D30A000AC8
:1024B700D2D320E8F1EFEEEBEDE5EDEE20F3F1EF0F
:1024C700E5F8EDEE210A000ACFF0E8EDFFF220CEA5
:1024D700D20A000ACFF0E8EDFFF220E7E0EFF0EED6
:1024E700F120ECE0F1F1E8E2E020D2D100202D204C
:1024F700EDE5F220E4E0EDEDFBF50A00202D20EEFE
:10250700F2E2E5F7E0FE0A000ACFF0E8EDFFF2207D
:10251700E7E0EFF0EEF120E3F0F3EFEFFB20D2D1AD
:1025270020000ACFF0E8EDFFF220E7E0EFF0EEF150
:1025370020E3F0F3EFEFFB20D2C8D220000ACFEE62
:10254700E2F2EEF020D2D320000AC4E0FE20D2D37C
:10255700E2EAEB20000ACAEEECE0EDE4E020D2D399
:1025670020000A5374617274210A000AD7F3E6EE59
:10257700E920E0E4F0E5F12120003E2A2C312CCFC0
:10258700E0F0E0ECE5F2F0FB20F1E8EDF5F0EEED40
:10259700EDEEE3EE20EFEEF0F2E00A003E4C2C42C7
:1025A70030312C256C752CD1EAEEF0EEF1F2FC20DF
:1025B700EEE1ECE5EDE02C35302C3130302C3230CB
:1025C700302C3330302C3630302C313230302C3206
:1025D7003430302C343830300A003E422C4731300A
:1025E7002C2562752CC8EDE2E5F0F1E8FF20EDE05F
:1025F70020EFF0E8B8ECE50A003E422C4731312CD9
:102607002562752CC8EDE2E5F0F1E8FF20EDE0204A
:10261700EFE5F0E5E4E0F7E50A003E422C4730320B
:102627002C2562752CD3EFF0E0E2EBE5EDE8E52031
:10263700EFEEF2EEEAEEEC2020285254532D4354ED
:1026470053290A003E532C4730332C256C752CC771
:10265700E0E4E5F0E6EAE020F1F2E0F0F2E020EF76
:10266700E5F0E5E4E0F7E828ECF1290A003E2A2C3A
:10267700312CCCEEF1F2EEE2EEE920EAEEEDF2F0EB
:10268700EEEBEBE5F020CACF2022C8F1E5F2FC2201
:102697002E20CFF0EEF2EEEAEEEB2000CAEEECEFE2
:1026A700E0F120D2CC312E312C00D2CC3132302C7B
:1026B7000020E8EDE8F6E8E0F2E8E2EDFBE92E0AB3
:1026C7000020E0E2F2EEEEEFF0E5E4E5EBE5EDE821
:1026D700E52E0A003E4C2C4B30392C256C752CD03E
:1026E700E5E6E8EC20F0E0E1EEF2FB2C30202D20CF
:1026F700E0E2F2EEEEEFF0E5E4E5EBE5EDE8E52C00
:1027070032202D20CAEEECEFE0F120E8EDE8F6E804
:10271700E0F2E8E2EDFBE92C33202D20D2CC313278
:102727003020E8EDE8F6E8E0F2E8E2EDFBE90A0040
:102737003E432C473130302C256C752CC4EEEFF31B
:10274700F1F2E8ECEEE520EAEEEBE8F7E5F1F2E28C
:10275700EE20ECEEE4F3EBE5E920D2C8D2343330D7
:102767000A003E432C473130302C256C752CC4EEC3
:10277700EFF3F1F2E8ECEEE520EAEEEBE8F7E5F14E
:10278700F2E2EE20ECEEE4F3EBE5E920D2D13433CC
:10279700300A003E532C4730342C2562752CCDEE81
:1027A700ECE5F020CACF0A003E4C2C4730392C25E7
:1027B7006C752CCAEEEDF42E20D2D32C3136202D99
:1027C70020EFF0FFECEEE520F3EFF02E2C33302076
:1027D7002D20F120E8F1EF2E20F0E5EBE52C31324A
:1027E70038202D20C1D0CF20C3F0E0EDE8F20A0059
:1027F7003E532C4B30352C2562752CD0E0E7ECE5A9
:10280700F020E3F0F3EFEFFB20D2C8D20A003E53EB
:102817002C4B31302C2562752CC0EAF2E8E2EDFB37
:10282700F520E3F0F3EFEF20D2C8D20A003E532C95
:102837004731372C25732CD0E5E2E5F0F1E8E2EDDE
:10284700FBE520D2C8D20A003E422C4B30362C255D
:1028570062752CC8EDE2E5F0F1E8FF20D2D10A005D
:102867003E422C4B30372C2562752CD0E5E2E5F043
:10287700F12028F0E0E7E2EEF0EEF22920D2D10ACB
:10288700003C21003C4230313D003C4731303D00A7
:102897003C4731313D003C4730323D003C47303307
:1028A7003D003C4730343D003C4730393D003C4B10
:1028B70030353D003C4B30363D003C4B30373D001A
:1028C7003C4B30393D003C4B31303D003C473137C4
:1028D7003D000008040C020A060E0109050D030B52
:0228E700070FD9
:1055D700526690000000000000000000000000007C
:0555E7000000000000BF
:10541200301A34E4906476F0906BAFE0FD906477DC
:10542200F090667BE0906478F0A37405F0906AAA2D
:10543200E0543FF063A20190647A63A201AF0512C7
:0A5442003757C21A7F01227F0022B3
:1053D700AE07906BC1E0FF30E10A6402F0906BC347
:1053E700E06429F0906BC1E0FF25E0F0906BC3E02B
:1053F700FD30E707906BC1E04401F0ED25E0906BCD
:0B540700C3F0EE30E704E04401F022A7
:0246E800AA071F
:1046EA00D233E4FB200205AF021253D79066D2E020
:1046FA00FF25E0F0EA30E709E04401F0A233B39283
:10470A0033906B2EE004F0E0B4081E9066D2E08588
:10471A001482851383F00514E51470020513906B57
:10472A00B0E004F0E4906B2EF0EA25E0FA0BBB0847
:10473A00B3200211A231303301B350047F808002CA
:10474A007F001253D79066D2E0FF25E0F0A232E450
:10475A0033600F14701B3031189066D2E04401F0B8
:10476A00800FA231303301B350079066D2E0440182
:10477A00F0906B2EE004F0200212906BC1E0FF3043
:10478A00E10A6402F0906BC3E06429F0906B2EE0BA
:10479A00B4081E9066D2E0851482851383F005144E
:1047AA00E51470020513906BB0E004F0E4906B2EF0
:0347BA00F0C20248
:0147BD0022D9
:02421000AA07FB
:10421200E4FB200238906BC1E0FF30E10A6402F057
:10422200906BC3E06429F0906BC1E0FF25E0F09051
:104232006BC3E0FE30E707906BC1E04401F0EE256E
:10424200E0906BC3F0EA30E704E04401F0906B2E9B
:10425200E004F0E024F8602914605A8000EA30E7B4
:104262000E906BC6E04401F0A207B392078007905C
:104272006BC6E054FEF0906BC6E0FF25E0F002430F
:1042820014EA30E70E906BC6E04401F0A207B39245
:10429200078007906BC6E054FEF0906BC6E0851174
:1042A20082851083F00511E51170020510906BAF45
:1042B200E004F0805D300926D21530141E906BC1E7
:1042C200E0FF30E10A6402F0906BC3E06429F090F1
:1042D2006BC3E0FF906BC1E04FFF227F00223007EB
:1042E20015EA20E724D209906BC6E0B42004D21468
:1042F2008017C2148013EA30E70FD209906BC6E030
:10430200B42004D2148002C214C202D207E4906B19
:104312002EF0EA25E0FA0BEB640860030242147FF8
:01432200009A
:014323002277
:02496400A907A1
:10496600E4906BB0F0906BC1F0906BC3F0302F0603
:104976007E667FA880047E6A7F818E358F367513AA
:104986006B75142F8F828E83E044C0F0E4906B2EFB
:10499600F0D202FCECC399501A853682853583E045
:1049A600FFC231C2321246E80536E53670020535D9
:1049B6000C80E1302F62D231C2327F201246E8E409
:1049C600FCE4FF1253D70CBC09F7906BC1E0FF3033
:1049D600E10A6402F0906BC3E06429F0906BC3E0D7
:1049E600FF30E003D38001C39230EFC313906BC353
:1049F600F0906BC1E030E009906BC3E04480F0803A
:104A060007906BC3E0547FF0D202906BC3E0FFA225
:104A1600309231D2321246E8D231C232E4FF124627
:074A2600E875136B75142FF6
:014A2D002266
:0100320022AB
:104A2E00E4FF0F2405F582E43461F5837405F00F7D
:104A3E0074052401F582E43461F583E4F0752901EF
:104A4E00752A66752B95FE782974FFF5F012109471
:104A5E00120E1CFDAC070F74052CF582E43461F5C3
:104A6E0083EDF00EBE04E0752901752A66752B994B
:104A7E00E4FE782974FFF5F0121094120E1CFDACB2
:104A8E00070F74052CF582E43461F583EDF00EBE4C
:104A9E0004E0752901752A66752B9DE4FE7829744C
:104AAE00FFF5F0121094120E1CFDAC070F74052CBE
:104ABE00F582E43461F583EDF00EBE04E075290154
:104ACE00752A66752BA1E4FE782974FFF5F0121095
:104ADE0094120E1CFDAC070F74052CF582E43461A4
:084AEE00F583EDF00EBE04E0BB
:014AF600229D
:0F562700C215C20AC209200003C20F22D20F22ED
:0B564100301905C2197F01227F0022F2
:03564C00C2AE22C9
:10560300EF540F9028D993FEC454F0FEEFC4540F07
:04561300932EFF22B1
:103A3400906BCE74FFF0A374B8F0E4906BCDF0906B
:103A44006BC4F0C217D21812343BE4F52BF52CE505
:103A54002C25E0FFE52B33FE74B12FF9746B3EFA8D
:103A64007B019069F91210ADE52C04120E84906963
:103A7400F91210A4900001E4120E96052CE52C70A6
:103A840002052B6408452B70C6E4F52BF52C74D085
:103A9400252CF582E4346BF5837401F0052CE52CB8
:103AA4007002052B452B70E674FC252CF582E4345A
:103AB40069F583E0FF7003023B88E52AC3748094B0
:103AC400814003023B88EFB4200A052CE52C7002E8
:103AD400052B80D474FC252CF582E43469F583E04D
:103AE400642D7031052CE52C7002052B24FCF9E4BF
:103AF4003469FA7B01C0031B8B32753300753400C3
:103B0400E4F535D003123BF78F29C3E529952AF54F
:103B1400290529802374FC252CF9E43469FA7B01F6
:103B2400C0031B8B32753300753400E4F535D003C4
:103B3400123BF78F2A752901E529D39400401974A3
:103B4400809481501374CF252AF582E4346BF58375
:103B5400E4F0052A152980E074FC252CF582E43470
:103B640069F583E0FF64207003023AACEF642D70C2
:103B740003023AACEF7003023AAC052CE52C700258
:103B8400052B80D4E4F52BF52CE51575F010A4FF76
:103B9400C3E52C9FE52B95F05052AE2BAF2C7C0047
:103BA4007D03120EB874F52FF974663EFA7B01900A
:103BB40066CF1210AD74D0252CF582E4346BF583F6
:103BC400E070047F2080027F009066CF1210A4EF83
:103BD400120E849066CF1210A4900001E4F5F01246
:103BE4000F18052CE52C7002052B809D12514212F2
:023BF4005398E4
:013BF60022AC
:105398007571C0C20EC20AE4F555C21AC216C2031C
:1053A800D219F567F56C906BC5F09069F6F0C211EB
:1053B8009066A5F0D238200804D20F800975121E15
:0F53C800906BC27401F0E4906A7FF01254862259
:022D58008F29C1
:102D5A00906004E024BE700302312A24FA70030250
:102D6A002FD5240460030231BF906005E054E324A8
:102D7A00807003022E94246060030231BF906007C2
:102D8A00E060030231BFA3E0640660030231BF9032
:102D9A006006E05407F51675F004A4FFAEF02404AB
:102DAA00FDE43EFCD3ED9408EC6480948040030279
:102DBA0031BF8E2B8F2CE52C25E0FFE52B33FE74DB
:102DCA00B12FF9746B3EFA7B019069F91210ADE4E8
:102DDA00F52A9069F91210A4900001120E35FF121B
:102DEA0056037409252AF582E43460F583E06F609E
:102DFA00179066A5E0B401109069F91210A4120E9A
:102E0A001C4440120E84D2119069F91210A4120EB9
:102E1A001C4480120E847409252AF582E43460F574
:102E2A0083E0FF1256039069F91210A4900001EF93
:102E3A00120E969069FAE475F002120ECA052AE596
:102E4A002AC39404408C90600EE0FE90600DE07CF2
:102E5A00002400FFEC3EFEE51625E0242AF582E474
:102E6A00346BF583EEF0A3EFF0302C17E51625E06E
:102E7A00242AF582E4346BAD82FC7E247F277B0210
:102E8A001244289066A57401F022906008E0640854
:102E9A0060030231BF906006E0FD75F004A42404CB
:102EAA00FFE435F0FED3EF9408EE6480948040038B
:102EBA000231BFED5407F516906010E0FE90600FE6
:102ECA00E07C002400FFEC3EFE906BD0F0A3EFF014
:102EDA00E51625E0242AF582E4346BF583E0FCA3A9
:102EEA00E0FDD39FEC9E4017ED2464FFE43CFED343
:102EFA00906BD1E09F906BD0E09E40030231BF30CF
:102F0A002C0D7E247F457C6B7DD07B02124428E504
:102F1A001625E0242AF582E4346BF583E475F00182
:102F2A00120ECA906007E0541FFF131313541FFDBB
:102F3A007C00E51675F004A4AEF02DF52CEC3EF5F8
:102F4A002BE52C25E0FFE52B33FE74B12FF9746BCA
:102F5A003EFA7B019069F91210AD906007E05407C0
:102F6A00752B00F52C752A80452B601AD3E52C9415
:102F7A0000E52B9400400FE52A13F52AE52C152CC1
:102F8A007002152B80E6906007E030E7179069F928
:102F9A001210A4E92401F9E43AFA120E1C452A1285
:102FAA000E8480189069F91210A4E92401F9E43A10
:102FBA00FA120E1CFFE52AF45F120E849069F912C8
:102FCA0010A4120E1C44C0120E8422302C0D7E2432
:102FDA007F5D7C607D067B01124428906007E0FDDE
:102FEA0030E6030231BF906006E075F020A4FFAE20
:102FFA00F0ED547F7C002FF52CEC3EF52BE5157592
:10300A00F010A4FFC3E52C9FE52B95F04003023195
:10301A00BF752F60753009AE2BAF2C7C007D031273
:10302A000EB874F52FF974663EFA7B019066CF12DA
:10303A0010AD906008E0FFC313752B00F52CE4F582
:10304A002AC3E52A952CE4952B40030231BF85302B
:10305A0082852F83E0752D00F52EA3E0FEE4252E50
:10306A00F52EEE352DF52DC3E52E9478E52D6480E9
:10307A00946C5006752DEC752E78D3E52E9488E560
:10308A002D648094934006752D13752E88AC2DAD52
:10309A002EEC120AC87B007A40799C7845120A26DF
:1030AA007B007AE079FF784412091D120B019066C1
:1030BA00CF1210A4900001EE8FF0120F18900001A9
:1030CA00120EE0FFAEF0C3EE64809480502A906640
:1030DA00CF1210A4EE5407F52D8F2E632EFF632D09
:1030EA0007052EE52E7002052D2400FFE52D34F884
:1030FA009000018FF0120F1874022530F530E43574
:10310A002FF52F9066CF1210A4120E1C44C0120E77
:10311A00849066D0E475F003120ECA052A02304B79
:10312A00906007E064037065906BCCE0605F302CC0
:10313A000B7E247F86E4FBFDFC124428906A7CE027
:10314A00FF906006E06F7040906BC9E0FF906009E5
:10315A00E06F703490657A7402F0A37408F0906A94
:10316A007CE090657CF0A3F0A37401F0E4A3F07F07
:10317A0006124AF7906AA97420F0302C0B7E247F3D
:10318A009BE4FBFDFC124428E4906BCCF0906007B2
:10319A00E064017020906AA9E0601A90600AE07009
:1031AA0002D201E4906AA9F0302C0A7E247FB6FB91
:0531BA00FDFC12442899
:0131BF0022ED
:104BA000E4F531E53175F002A424B1F9746B35F008
:104BB000FA7B019069F91210AD120E1CFF30E670FD
:104BC0009069F91210A4EF54BF120E847B017A6A27
:104BD00079818B328A338934906BCBE0120E8474E6
:104BE000012534F534E43533F533300616E5312448
:104BF00091AB32AA33A934120E84C22F7F0212491C
:104C0000648029AB32AA33A9347490120E847401E3
:104C10002534F534E43533F533E53104AB32AA33CA
:104C2000A934120E84C22F7F03124964D203D32207
:0D4C30000531E531C394085003024BA3C3C6
:014C3D002254
:10544C00EF75F003A424F5F9746635F0FA7B01903E
:10545C0066CF1210ADE4FFEFC39515501B9066CFCD
:10546C001210A4120E1C30E702D3229066D0E47501
:09547C00F003120ECA0F80DFC319
:015485002204
:10118C00EF24F0700302148324C0602624E0700363
:10119C000216BC24E0700302137A24B0700302160A
:1011AC00BC24F0606080003008030218A5D238D24D
:1011BC000F22302C0B7E247FCEE4FBFDFC12442846
:1011CC00124BA050030218A57B017A6A79818B2BF4
:1011DC008A2C892D906BCBE0120E847401252DF591
:1011EC002DE4352CF52CAB2BFAA92D7450120E8452
:1011FC007401252DF52DE4352CF52CC22F7F021210
:10120C004964D20322302C0B7E247FDAE4FBFDFCF4
:10121C001244287B017A6B79B19069F91210AD30C8
:10122C0006647530FFE4F52EF52F9069F91210A4C1
:10123C00120E1CFF30E710E53030E705852F3080AB
:10124C0006EF4440120E849069FAE475F002120E17
:10125C00CA052FE52F7002052E6408452E70CBE5CC
:10126C003030E7177F64125636202C030218A57E07
:10127C00247FF4E4FBFDFC12442822E530249190F9
:10128C006AABF002137A9066A5E070177F64125671
:10129C0036202C030218A57E247FF4E4FBFDFC12FF
:1012AC004428227A6679A8752B01752C66752DA8B1
:1012BC00906BCBE0AB2BAA2CA92D120E84740125BC
:1012CC002DF52DE4352CF52CAB2BFAA92D74F01241
:1012DC000E847401252DF52DE4352CF52CAB2BFA51
:1012EC00A92D7408120E847401252DF52DE4352CCE
:1012FC00F52CE4F52EF52F301D129069F91210A47F
:10130C00900001120E35FF125603800D9069F912F0
:10131C0010A4900001120E35FF8F30301E06E53000
:10132C00F4FF8002AF30AB2BAA2CA92DEF120E8448
:10133C009069FAE475F002120ECA7401252DF52D90
:10134C00E4352CF52C052FE52F7002052EC39408DF
:10135C00E52E940040A1D22F7F0B124964302C0B48
:10136C007E257F03E4FBFDFC124428D20322906A05
:10137C00ABE0540F6004D2068002C206302C0D7E06
:10138C00257F0F7C6A7DAB7B0212442830061690B9
:10139C006AABE0540F75F002A424AFF9746B35F00E
:1013AC00FA7B018012906AACE075F002A424AFF9CC
:1013BC00746B35F0FA7B019069F91210AD7A66798D
:1013CC00A8752B01752C66752DA8906BCBE0AB2BFB
:1013DC00AA2CA92D120E847401252DF52DE4352C83
:1013EC00F52C906AABE0AB2BAA2CA92D120E8474B1
:1013FC0001252DF52DE4352CF52C752E00752F03BC
:10140C00200620906AACE0AB2BAA2CA92D120E84DE
:10141C007401252DF52DE4352CF52C052FE52F70B9
:10142C0002052E301D129069F91210A490000112C1
:10143C000E35FF125603800D9069F91210A490001E
:10144C0001120E35FF8F30301E06E530F4FF80029E
:10145C00AF30AB2BAA2CA92DEF120E84AF2FD22FAD
:10146C00124964D203202C030218A57E257F03E4C5
:10147C00FBFDFC12442822906AABE0540F6004D2AE
:10148C00068002C206302C0D7E257F297C6A7DAB3E
:10149C007B0212442830060E906AABE0540F148580
:1014AC0015F0A4FF800A906AACE0148515F0A4FF37
:1014BC00752E008F2FE51575F010A4FFC3E52F9F37
:1014CC00E52E95F040030218A5AF2F12544C401294
:1014DC00202C030218A57E247FF4E4FBFDFC1244AF
:1014EC002822AE2EAF2F7C007D03120EB874F52F80
:1014FC00F974663EFA7B019066CF1210AD7A66796C
:10150C00A88B2B752C66752DA8906BCBE0AB2BAAFA
:10151C002CA92D120E847401252DF52DE4352CF5F6
:10152C002C906AABE0AB2BAA2CA92D120E84740163
:10153C00252DF52DE4352CF52C75300220061A904E
:10154C006AACE0AB2BAA2CA92D120E847401252DAC
:10155C00F52DE4352CF52C0530E4F52EF52FC3E5EF
:10156C002F9515E52E940040030216A420060302C5
:10157C0016509066CF1210A4120E1C30E568900025
:10158C0001120EE0FFE5F05407FCAD07120AC8E4A7
:10159C00FBFAF97845120A26E4FBFA79FA7842123A
:1015AC00091D120B01AB2BAA2CA92DEF120E849046
:1015BC0066CF1210A4900001120EE0E5F030E30E9D
:1015CC00AB2BAA2CA92D120E1CF404120E84AB2BDF
:1015DC00AA2CA92D747D120E627401252DF52DE413
:1015EC00352CF52C805A9066CF1210A49000011265
:1015FC000EE0C3E5F064809480500F782BE475F016
:10160C0001121094E4120E8480369066CF1210A44E
:10161C00900001120EE0FDACF0EC120AC8E4FBFAEB
:10162C00F97845120A26E4FBFA797A784312091DF7
:10163C00120B01782BE475F001121094EF120E844A
:10164C000530803F9066CF1210A4900001120EE07E
:10165C00FF782BE475F001121094EF120E84906653
:10166C00CF1210A4900001120EE0E5F0540FFF33DE
:10167C0095E0782BE475F001121094EF120E8405AE
:10168C003005309066D0E475F003120ECA052FE5D4
:10169C002F7002052E02156AD22FAF30124964301A
:1016AC002C0B7E257F03E4FBFDFC124428D2032285
:1016BC00906AABE0FF540F6004D2068002C2069021
:1016CC006A7FE07003021874E4F09066F4E06F60D7
:1016DC00030218A5906AACE0FF9066A3E06F60036C
:1016EC000218A5906AADE0FF9066A6E06F60030259
:1016FC0018A5302C0A7E257F44FBFDFC12442830B3
:10170C000618906AABE0540F1475F008A4FF9069AA
:10171C00F8E0FEEF8EF084FF8014906AACE0147554
:10172C00F008A4FF9069F8E0FEEF8EF084FF906A59
:10173C007CEFF030061A906AABE0540F14C454F0EE
:10174C00FF9069F8E025E0FEEF8EF084AFF0801694
:10175C00906AACE014C454F0FF9069F8E025E0FE08
:10176C00EF8EF084AFF0906BC9EFF09066F4E0541C
:10177C00F0FFBFE006906BC9E004F0300607906AFA
:10178C00ACE0FF8005906AADE0FFE4F530EF20E0BF
:10179C0012906BC9E02402F0EFC313FF0530E53063
:1017AC00B408EA90657A7442F0A37418F0906A7CDD
:1017BC00E090657CF0906BC9E090657DF0A37401BE
:1017CC00F0E4A3F07F06124AF7906BCC740AF07F1A
:1017DC0014125636302C0D7E257F507C657D7A7B1D
:1017EC00061244287B017A6A79818B2B8A2C892DED
:1017FC00906BCBE0120E847401252DF52DE4352C65
:10180C00F52C752E00752F012006539066F4E0AB75
:10181C002BAA2CA92D120E847401252DF52DE4353F
:10182C002CF52C9066A3E0AB2BAA2CA92D120E84C0
:10183C007401252DF52DE4352CF52C9066A6E0AB26
:10184C002BAA2CA92D120E847401252DF52DE4350F
:10185C002CF52C7403252FF52FE4352EF52EAF2FF8
:10186C00C22F124964D20322906A7F7496F0906A58
:10187C00ABE09066F4F0906AACE09066A3F0906AEE
:10188C00ADE09066A6F0302C107E257F5C7C6A7DE6
:09189C00AA906BAFE0FB12442896
:0118A5002220
:1031C000302112C221906A7FE0600214F09069F60B
:1031D000E0600214F0302D15200812C22D906BCC47
:1031E000E0600214F0906AA9E0600214F0300E2D45
:1031F000C3E5549570FFE553956FFED3EF9440EE11
:10320000940040197B087D40AF70AE6F1247BEE559
:10321000702440FFE4356F540FF56F8F7030181035
:10322000125398C2187E257F69E4FBFDFC124428E6
:103230003008030232F1200A030232C3E56C54382D
:1032400065677003023387E56724085438F5671310
:103250001313541F2457F8E6906A80F0200915E0F4
:10326000FF1242107529008F2A906BAFE0D3948033
:1032700040CA8033C291C215C20AC209C20F906A05
:10328000AAE0543F752900F52A906BCBE0B52A17C8
:10329000E4B52913906AABE054F0FF12118C2003BF
:1032A0009BD238D20F8095302C0D7E257F727C6AA0
:1032B0007DAA7B01124428D20FE4F555D238D2B151
:1032C00002323C200F03023387303803023387D2A7
:1032D00091D20AE4906BAFF0906BC3F0906BC1F0A9
:1032E000D207D202906B2EF075106A7511AA0233C4
:1032F00087202D03023387C22D1512E512706075E9
:10330000121E30160302338720037C906BC2E070DC
:1033100012906AAB74F0F0FF12118C906BC2E00453
:10332000F08064906AAB7410F030060FE0FF906B91
:10333000C2E0FEEF4E906AABF08008906BC2E09066
:103340006AACF07F1012118C906BC2E004F0906BAD
:10335000C7E0FF906BC2E0D39F402CE4F0802820B0
:103360001625200322124BA0501D906A81E0906A1E
:10337000AAF0906A82E0906AABF0906A83E0906A6B
:10338000ACF07F9012118C301661E56D6568604D70
:10339000E56D24085438FFE56854386F60047E01F9
:1033A00080027E00906BB0E060047D0180027D00B1
:1033B000EE5D700302343A851482851383E0FEE5E6
:1033C0006D131313541F245FF8A6068F6D0514E5C3
:1033D0001470020513906BB0E014F080B3C216D2E3
:1033E000B1200804D238D20FC2902230034C30B141
:1033F0000B3013089066A4E09069F6F0C2B1301368
:103400000930B0069069F6E0703085148285138328
:10341000E0FFE56D131313541F245FF8A607E56D55
:1034200024085438F56D0514E51470020513906BEB
:0A343000B0E014F0C203D216D290EF
:01343A00226F
:10386500906BCDE0601EA3E0FEA3E0FFC3E49FFFE5
:10387500E49EFEAB07FAE4F9F8FF7EC27D01FC1277
:103885005354801E906BCEE0FEA3E0FFC3E49FFF80
:10389500E49EFEAB07FAE4F9F87F207E1CFDFC12DE
:1038A50053548F318E308D2F8C2E7BFF7A25798165
:1038B50012294B7BFF7A2579A385313885303785E9
:1038C5002F36852E3512294B7BFF7A2579E1A20DFE
:1038D500E433F53512294B7BFF7A267900A20BE4F8
:1038E50033F53512294B7BFF7A267921A213E43370
:1038F500F53512294B7BFF7A26794B9066A4E07546
:10390500F00AA4FFAEF0E48F388E37F536F53512A0
:10391500294B7535FF7536267537747B017A6B79BA
:10392500D01229452006147535FF7536267537A33F
:103935007B017A6B79D01252B380127535FF7536DB
:10394500267537B17B017A6B79D01252B3300814E2
:103955007535FF7536267537B87B017A6B79D012C8
:1039650052B380127535FF7536267537C87B017AD7
:103975006B79D01252B37B017A6B79D012294B7BCC
:10398500FF7A2679DBE4851738F537F536F53512F4
:10399500294B7BFF7A277937E4753804F537F536F7
:1039A500F53512294B7BFF7A277969E4753802F5DD
:1039B50037F536F53512294B7BFF7A27799A906BC7
:1039C500CBE0F53512294B7BFF7A2779AF9069F863
:1039D500E0FFE48F38F537F536F53512294B7BFFD7
:1039E5007A2779F785153512294BE51730E10F7BD5
:1039F500FF7A287915906BC7E0F53512294B753597
:103A0500017536697537FC7BFF7A28793412294BA5
:103A15007BFF7A28794FA21EE433F53512294B7BBB
:0E3A2500FF7A287967A21DE433F53512294B8C
:013A33002270
:10343B007E287F88124DDEEF4E70037F01227E289F
:10344B007F8B124DDEEF4E60711251A0906CD0123B
:10345B001057E4FFFEFDFC906CD012104BC3121002
:10346B002E6020906CD012104BE47F207E1CFDFC54
:10347B00120F8E121020906BCEEEF0A3EFF0E490B3
:10348B006BCDF0E47FB07E04FDFC906CD012104B42
:10349B00D312102E4033906BCD7401F0906CD01280
:1034AB00104B7F007EC27D017C00120F8E1210200C
:1034BB00906BCEEEF0A3EFF0800F906BCE74FFF01D
:1034CB00A374B8F0E4906BCDF07E287F91124DDEA3
:1034DB00EF4E600C1255EDEF24D024FF920D8002BD
:1034EB00C20D7E287F97124DDEEF4E600C1255ED0C
:1034FB00EF24D024FF920B8002C20B7E287F9D12FB
:10350B004DDEEF4E600C1255EDEF24D024FF9213DD
:10351B008002C2137E287FA3124DDEEF4E60131282
:10352B0051A0E47B0AFAF9F8120F8E9066A4EFF023
:10353B008005E49066A4F07E287FA9124DDEEF4E45
:10354B00600A1251A0906BCBEFF08006906BCB749E
:10355B0001F07E287FAF124DDEEF4E600A1251A0B4
:10356B009069F8EFF080069069F87410F07E287F70
:10357B00B5124DDEEF4E60071251A08F158003750B
:10358B0015087E287FBB124DDEEF4E600C1255EDF9
:10359B00EF24D024FF921E8002C21E7E287FC11210
:1035AB004DDEEF4E600C1255EDEF24D024FF921D33
:1035BB008002C21D7E287FC7124DDEEF4E600712C0
:1035CB0051A08F178003E4F517E51720E103C380A3
:1035DB0001D39208E51720E003C38001D392067E46
:1035EB00287FCD124DDEEF4E60081251A0906BC7B5
:1035FB00EFF0906BC7E0D3941040037410F07E286B
:10360B007FD3124DDEEF4E6047E4F52D1255ED8F53
:10361B002EE52E643C6039AF2D052D74FC2FF58201
:10362B00E43469F583E52EF01255ED8F2EE52E640B
:10363B003C6007E52DC3948040DDE52DB480021579
:10364B002D74FC252DF582E43469F583E4F0801E9E
:10365B00AF2D052D74FC2FF582E43469F5837420AE
:10366B00F074FC252DF582E43469F583E4F07F00DA
:01367B00222C
:10091D00EC4D6011E8497017ED33EC3304600DE4D4
:10092D00FCFFFEFD22E933E8330470F8020B6D1273
:10093D000B3858046009E4CC248150062850090274
:10094D000B77284003020B74C0E0EB4A7044B9806A
:10095D0006D0E0FB020B63EF4E701CBD8008EBFF71
:10096D00EAFEE9FD80EBE98DF0A4FEE5F0020A0652
:10097D00E9CDF9EAFEEBFFEF89F0A4FCE5F0CE89B5
:10098D00F0A42EFFE435F0CD89F0A42DFEE435F072
:10099D008067EF4E7005BD80D780C3EF8BF0A4ACA0
:1009AD00F0EE8BF0A42CFCE435F0F8EF8AF0A42CDB
:1009BD00E5F038FCE433CB8DF0A42CFCE5F03BF8EE
:1009CD00EE8AF0A42CFCE5F038F8E433CF89F0A4DE
:1009DD002CFCE5F038CF3400CE89F0A42FFFE5F0E4
:1009ED003EFEE433C98DF0A42EFEE5F039CD8AF03C
:1009FD00A42FFFE5F03EFEE43DFD33D0E0FB5007B4
:100A0D000BBB000F020B77EC2CFCEF33FFEE33FE2C
:060A1D00ED33FD020B4F5A
:100A2300020B77EC5D046005E859047003020B6D5B
:100A3300120B38580460F6EC4860F2EC7004FDFECB
:100A4300FF22C860DB2481C85009C39860025006A6
:100A5300020B749850CAF582E9294B4A7005AB82A0
:100A6300020B6375F0007C1A7880C3EF9BEE9AED5E
:100A730099400DC3EF9BFFEE9AFEED99FDE842F01E
:100A8300DC23ACF0D0E0FFD0E0FED0E0FDAB822071
:100A9300E7101BEB60BAEC2CFCEF33FFEE33FEEDFB
:100AA30033FD020B4FE803F830E705C0F075F000A3
:100AB300EF2FFFEE33FEED33FD40B830E7C280AADF
:100AC30075F020800E75F010800575F0087D007EAE
:100AD300007F003392D530D503121020EC33401041
:100AE300EF33FFEE33FEED33FDEC33FCD5F0ED22B7
:0E0AF300E5F0247EA2D513CC92E7CDCEFF22F3
:100B0100EDD2E7CD33EC3392D524814006E4FFFEEC
:100B1100FDFC22FCE4CFCECDCC24E0501174FF804B
:100B2100EDC3CC13CCCD13CDCE13CECF13CF0470E8
:070B3100F030D5DE021020B8
:1028E900E5492435F8E6054922783230360278354B
:1028F900E475F001121094020E1C202FEB7F2ED2EA
:102909002F8018EF540F2490D43440D4FF30330B68
:10291900EF24BFB41A0050032461FFE54A60021591
:102929004A054DE54D7002054C30360D7832E47597
:10293900F001121094EF020E8402530B7403D23685
:102949008003E4C236F5498B328A338934E4F54A87
:10295900F54CF54DE54A60077F2012292480F5756D
:102969004BFFC230C22FC231C232C234C235C23764
:102979001228F2FF700D3036057F00122935AF4D50
:10298900AE4C22B4255FC2D5C2331228F2FF24D03F
:10299900B40A00501A75F00A784A30D50508B6FF0E
:1029A9000106C6A426F620D5047002D23280D924A5
:1029B900CFB41A00EF5004C2E5D233022C22D23030
:1029C90080C6D22F80C0D23180BCD2D580BAD23451
:1029D90080B47F201229242031077401B54A0040B0
:1029E900F11228E9FF12292402295DD237D2358054
:1029F900951228E9FB1228E9FA1228E9F94A4B70DD
:102A09000679197A2D7BFF20312EE54A602A7E004E
:102A19008E82758300120E3560060EEE654B70F0DE
:102A2900C2D5EBC0E0EAC0E0E9C0E0EE122C82D0EA
:102A3900E0F9D0E0FAD0E0FB120E1CFF60AAEBC06F
:102A4900E0EAC0E0E9C0E0122924D0E02401F9D08D
:102A5900E03400FAD0E0FBE54B0460DCD54BD980CB
:102A690087D23180A2122C6560F7E54B7001041200
:102A79000B82A94B600DE54B600914F54B122D0C27
:102A8900EF60F3EA30E702F404C3995077EAF425DA
:102A99004B0430E701E404F54B800D122C6560C14D
:102AA900EA054B254B120B82EA7848F630E701E438
:102AB900254B04D54B0420340114122C82E4C0E0C8
:102AC900122D0C7848E6601320E70714F612290C3A
:102AD900802204F6D0E014C0E07F0012290CE54BF7
:102AE9006007122903154B800B303403122903D0D8
:102AF900E002295DD0E00480C5122C6560A0E54B99
:102B090004120B827848EAF6E54B2034026001048E
:052B19002404122C82CF
:102B1E0074FF04C0E0122D0C12290CE54B20340278
:102B2E006003122903D0E0B54BE87F4512291678D1
:102B3E0048E67F2B30E7047F2DF404C0E0122924F1
:102B4E00D0E075F00A84C0F012290DD0E012290DE4
:102B5E0002295D791080027908C235C2378008D209
:102B6E00D5790A8004790AC2D5E54B047002F54B7B
:102B7E00E4FAFDFEFF1228E9FC7B08203013122830
:102B8E00E9FD7B10302F0A1228E9FE1228E9FF7B9F
:102B9E0020EC3382D592D55013C3E4302F069FFF1D
:102BAE00E49EFEE42030039DFDE49CFCE4CBF8C2E1
:102BBE0030EC700CCFCECDCCE824F8F870F3801743
:102BCE00C3EF33FFEE33FEED33FDEC33FCEB33FBA3
:102BDE00994002FB0FD8E9EB303005F8D0E0C4483D
:102BEE00B230C0E00AEC4D4E4F78207B0070C2EA46
:102BFE00B54B0040BCC0E0122C84D0F0D0E02030A9
:102C0E0004C4C0E0C4B230C0F012290DD0F0D5F02B
:102C1E00EB02295D1210B629FA532B615829CB4CC1
:102C2E0029C7422B654F2B6D442B6D4929E0432B51
:102C3E0073552AA4462B02452A6E472D395029CFAB
:102C4E002D29D32E29F62B29D72329F4202D222AFC
:102C5E00298F48000029EEE54BB4FF03754B061291
:102C6E0028E9FC1228E9FD1228E9FE1228E9FF786E
:102C7E0041020BB1790AA2D5203214303409B910B1
:102C8E00020404B9080104A2D52035025001042023
:102C9E0031689231B54A005034C0E07F203032198D
:102CAE007F30A23172357234500F122CDBC231C21A
:102CBE0035C234C2377F30800F303403E9C0E012A2
:102CCE002924303403D0E0F9D0E0B54ACC303417A3
:102CDE007F30B9100C1229247F583033077F78804B
:102CEE0003B908031229243031057F2D0229247FD0
:102CFE00202037F87F2B2035F322923180CF7F00B2
:102D0E00B4070050052441F8E6FF22286E756C6C5E
:102D1E002900D2301228E93030F8C230784A30D546
:102D2E000108F602298F2D504349581228E9240331
:102D3E00B405004001E4902D3493122915743A1213
:0A2D4E002915D232754A04022B61E8
:100B3800E9D2E7C933E833F892D5EDD2E7CD33EC03
:070B480033FC5002B2D5227C
:100B4F00EC30E7100FBF000C0EBE00080DBD000407
:100B5F000BEB6014A2D5EB13FCED92E7FD2274FFB3
:100B6F00FCFDFEFF22E480F8A2D574FF13FC7D800C
:030B7F00E480EF20
:100B8200F920E72824F950037907E4F42402FB183A
:100B9200DBFDE624FB5014E9600DE4F618E604F6EA
:0F0BA200B40A08E4F6D9F57401F60A22C2D52286
:100BB100ED33EC3392D5FA602AB4FF33EDC2E77B13
:100BC100FF60067A0B79D6E4227A0B79DF20D5040F
:100BD1007A0B79DA224E614E002B494E46002D499F
:100BE1004E4600E47A08F608DAFC7B00740722E836
:100BF100C0E0ECC0E0EDC0E0EEC0E0EFC0E0EA75BF
:100C0100F010A4CAABF075F04DA42BFBE435F0FC59
:100C1100EA2410FAEB34C5FBEC34D9FCEDC2E7FF52
:100C210075F056A4F42411C5F0F434C58FF0A42A4C
:100C3100E5F03BE43CF620E714120DDCD0E0FFD0F8
:100C4100E0FED0E0FDD0E0FC120A268014F404128C
:100C51000DDCD0E0FFD0E0FED0E0FDD0E0FC1209D9
:100C61001DD0E0F8E6FAEDD2E7CD33EC332482FB78
:100C7100E4C3CF33CFCE33CECD33CD33DBF37B07DC
:100C810075F00A846004F6081B0AE5F0F6088FF097
:100C9100740AA4FFACF08EF0740AA42CFEACF050E0
:100CA100010C8DF0740AA42CFDE435F0F608DBDEAE
:030CB100740722A3
:100CB400020B6DE86480F8E933E83360110460F0F6
:100CC400ED33EC337009E8FCE9FDEAFEEBFF2204A6
:100CD40060DED3EB9FEA9EE99DE8C2E78CF0C2F7A1
:100CE40095F0400CE8CCF8E9CDF9EACEFAEBCFFB6D
:100CF400120B3885D0F05804700320D5B3E8047083
:100D0400075002B2D5020B7792D5EC0460F7E4CC1D
:100D1400C0E0C398F8603B94186008400DD0E0FB35
:100D2400020B4FE4FBFAC9FC8028E830E406E4C96E
:100D3400FBE4CAFCE830E305E4C9CACBFCE8540789
:100D44006010F8C3E913F9EA13FAEB13FBEC13FC94
:100D5400D8F130F52FC3E49CFCEF9BFFEE9AFEED37
:100D640099FDD0E0FBEF4E4D4C701222DB03020BD9
:100D740074EC2CFCEF33FFEE33FEED33FDED30E786
:100D8400EB020B4FEF2BFFEE3AFEED39FDD0E0FB0B
:100D940050130BBB0003020B77ED13FDEE13FEEFB4
:080DA40013FFEC13FC020B4FDE
:100DAC003F8000004120000042C80000447A00004F
:100DBC00461C400047C35000497424004B189680D1
:100DCC004CBEBC205A0E1BCA6753C21C749DC5AEC8
:100DDC00FB60065407601C2323120E0AEB54386088
:100DEC0009120DF6120E0512091DECF8EDF9EEFACA
:100DFC00EFCB22EB120E0580F1543803241C900D1E
:100E0C00ACFE93FC0EEE93FD0EEE930ECE93FF22F2
:104CDA000218A6E493A3F8E493A34003F68001F232
:104CEA0008DFF48029E493A3F85407240CC8C333DB
:104CFA00C4540F4420C8834004F456800146F6DFAA
:104D0A00E4800B01020408102040809055D1E47E13
:104D1A00019360BCA3FF543F30E509541FFEE4939E
:104D2A00A360010ECF54C025E060A840B8E493A365
:104D3A00FAE493A3F8E493A3C8C582C8CAC583CA90
:104D4A00F0A3C8C582C8CAC583CADFE9DEE780BE48
:0155EC0000BE
:100E1C00BB010689828A83E0225002E722BBFE02D4
:090E2C00E32289828A83E4932207
:100E3500BB010CE58229F582E5833AF583E0225072
:100E450006E92582F8E622BBFE06E92582F8E222BC
:0D0E5500E58229F582E5833AF583E49322D6
:100E6200BB010989828A83F8E028F022500327F720
:100E720022BBFE05F8E328F3228A838982F8E493F1
:020E8200282224
:100E8400BB010689828A83F0225002F722BBFE014D
:020E9400F32247
:100E9600F8BB010DE58229F582E5833AF583E8F092
:100EA600225006E92582C8F622BBFE05E92582C83E
:020EB600F22226
:100EB800EF8DF0A4A8F0CF8CF0A428CE8DF0A42E4E
:020EC800FE2208
:100ECA00C5F0F8A3E028F0C5F0F8E58215827002B3
:060EDA001583E038F02250
:100EE000BB0110E58229F582E5833AF583E0F5F050
:100EF000A3E0225009E92582F886F008E622BBFE2D
:100F00000AE92582F8E2F5F008E222E5832AF58372
:080F1000E993F5F0A3E9932237
:100F1800F8BB0111E58229F582E5833AF583E8F00B
:100F2800E5F0A3F0225009E92582C8F608A6F022C8
:0D0F3800BBFE09E92582C8F2E5F008F222AF
:0D0F4500EF2BFFEE3AFEED39FDEC38FC22FB
:100F520075F008758200EF2FFFEE33FECD33CDCC56
:100F620033CCC58233C5829BED9AEC99E5829840D9
:100F72000CF582EE9BFEED9AFDEC99FC0FD5F0D6B6
:100F8200E4CEFBE4CDFAE4CCF9A88222B800C1B9E0
:100F92000059BA002DEC8BF084CFCECDFCE5F0CB1E
:100FA200F97818EF2FFFEE33FEED33FDEC33FCEB57
:100FB20033FB10D703994004EB99FB0FD8E5E4F912
:100FC200FA227818EF2FFFEE33FEED33FDEC33FCFF
:100FD200C933C910D7059BE99A4007EC9BFCE99AF3
:100FE200F90FD8E0E4C9FAE4CCFB2275F010EF2F38
:100FF200FFEE33FEED33FDCC33CCC833C810D70738
:101002009BEC9AE899400AED9BFDEC9AFCE899F872
:0E1012000FD5F0DAE4CDFBE4CCFAE4C8F92205
:10535400C2D5E830E70FB2D5E4C39BFBE49AFAE484
:1053640099F9E498F8EC30E717B2D512538A120F82
:105374008EE4C39BFBE49AFAE499F9E498F8800379
:10538400120F8E30D50DE4C39FFFE49EFEE49DFD15
:04539400E49CFC2277
:0E102000C3E49FFFE49EFEE49DFDE49CFC22E1
:10102E00EB9FF5F0EA9E42F0E99D42F0E89C45F018
:01103E00228F
:0C103F00E0FCA3E0FDA3E0FEA3E0FF2224
:0C104B00E0F8A3E0F9A3E0FAA3E0FB2228
:0C105700ECF0A3EDF0A3EEF0A3EFF0220C
:10106300A8828583F0D083D08212107A12107A126C
:10107300107A12107AE473E493A3C583C5F0C58391
:10108300C8C582C8F0A3C583C5F0C583C8C582C8D7
:01109300223A
:10109400FAE6FB0808E6F925F0F618E6CA3AF6225D
:0910A400E0FBA3E0FAA3E0F9224D
:0910AD00EBF0A3EAF0A3E9F02244
:1010B600D083D082F8E4937012740193700DA3A3C9
:1010C60093F8740193F5828883E4737402936860DD
:0610D600EFA3A3A380DFDD
:1052B3008B328A3389348B388A39893AAB32053455
:1052C300E534AA337002053314F9120E1C70ED7421
:1052D300FF2534F53474FF3533F533AB350537E546
:1052E30037AA367002053614F9120E1CFFAB3205CD
:1052F30034E534AA337002053314F9EF120E8470C7
:08530300DAAB38AA39A93A22FD
:103BF7008B2F8A308931E4F53BF53AF539F538F5FD
:103C070036F537E533453445326012EBC0E0EAC09C
:103C1700E0E9C0E0AB32AA33A93412112BAB2F0570
:103C270031E531AA307002053014F9120E1CF53C4B
:103C3700C394094007E53CD3940D40E1E53C64207B
:103C470060DBE53CB42D054337038016E53CB42B18
:103C570005433701800C74FF2531F53174FF35308A
:103C6700F530E53560046410703FAB2FAA30A931F9
:103C7700120E1C64306009E535702E75350A8029EF
:103C8700900001120E35FF64786004EFB4581343B7
:103C9700370175351074022531F531E43530F530CB
:103CA7008007E5357003753508AB2F0531E531AA77
:103CB700307002053014F9120E1CF53CC3946140B4
:103CC7000AE53CD3947A5003533CDF74D0253CF586
:103CD7003CC3940A400CE53C9411406D74F9253CB3
:103CE700F53CE53CD395355060433701853B40852E
:103CF7003A3F85393E85383DAF357E00E4FCFDAB64
:103D07003BAA3AA939A8381210DCC8ECC8C9EDC9D2
:103D1700CAEECACBEFCBE4FCFDFEEB253CF53BEE50
:103D27003AF53AED39F539EC38F538AF3BAE3AADFF
:103D370039FCAB40AA3FA93EA83DD312102E500331
:103D4700023CB0433704023CB0E53720E003E4808F
:103D57002DE53345344532601EAB2FE53124FFF99D
:103D6700E53034FFFAEBC0E0EAC0E0E9C0E0AB328F
:103D7700AA33A93412112BE53730E20774FFFFFE8F
:103D8700FDFC22E537AF3BAE3AAD39AC3830E10345
:043D970002102022D4
:1010DC00E88FF0A4CC8BF0A42CFCE98EF0A42CFCB3
:1010EC008AF0EDA42CFCEA8EF0A4CDA8F08BF0A431
:1010FC002DCC3825F0FDE98FF0A42CCD35F0FCEB90
:10110C008EF0A4FEA9F0EB8FF0A4CFC5F02ECD3954
:0F111C00FEE43CFCEAA42DCE35F0FDE43CFC22C1
:10112B00BB011A89828A83D0F0D0E0F8D0E0F9D0E5
:10113B00E0FAD0E0FBE8C0E0C0F00210AD5016E9D9
:10114B00F8D083D082D0E0F9D0E0FAD0E0FBC082B7
:10115B00C08302117ABBFE16E9F8D083D082D0E0AF
:0F116B00F9D0E0FAD0E0FBC082C08302118322EA
:09117A00EBF608EAF608E9F6229A
:09118300EBF208EAF208E9F2229D
:00000001FF
